:100000000110060000000000A01B0000FF0000001F
:10001000020BB9751AFF22FFFFFFFF0214E67E05EF
:1000200090008CE06F6007EFF0E490008FF090009C
:100030008CE07001FE90008FE004F0C39E50037FBF
:10004000002290008F7405F07F0122021676E4FBF7
:10005000EB25E025E02480F8120232EB25E025E0D4
:10006000248CF812024B0BBB03E622021004BB01E6
:100070000689828A83E0225002E722BBFE02E32245
:1000800089828A83E49322EF8DF0A4A8F0CF8CF0CC
:10009000A428CE8DF0A42EFE22BC000BBE0029EFBA
:1000A0008DF084FFADF022E4CCF875F008EF2FFF5F
:1000B000EE33FEEC33FCEE9DEC984005FCEE9DFE2D
:1000C0000FD5F0E9E4CEFD22EDF8F5F0EE8420D274
:1000D0001CFEADF075F008EF2FFFED33FD400798E3
:1000E0005006D5F0F222C398FD0FD5F0EA22E88F32
:1000F000F0A4CC8BF0A42CFCE98EF0A42CFC8AF0AC
:10010000EDA42CFCEA8EF0A4CDA8F08BF0A42DCCAD
:100110003825F0FDE98FF0A42CCD35F0FCEB8EF006
:10012000A4FEA9F0EB8FF0A4CFC5F02ECD39FEE4EC
:100130003CFCEAA42DCE35F0FDE43CFC2275F00831
:10014000758200EF2FFFEE33FECD33CDCC33CCC51F
:100150008233C5829BED9AEC99E58298400CF5823A
:10016000EE9BFEED9AFDEC99FC0FD5F0D6E4CEFBAC
:10017000E4CDFAE4CCF9A88222B800C1B90059BA9A
:10018000002DEC8BF084CFCECDFCE5F0CBF97818C8
:10019000EF2FFFEE33FEED33FDEC33FCEB33FB10C2
:1001A000D703994004EB99FB0FD8E5E4F9FA2278DC
:1001B00018EF2FFFEE33FEED33FDEC33FCC933C9EE
:1001C00010D7059BE99A4007EC9BFCE99AF90FD8F8
:1001D000E0E4C9FAE4CCFB2275F010EF2FFFEE3318
:1001E000FEED33FDCC33CCC833C810D7079BEC9A57
:1001F000E899400AED9BFDEC9AFCE899F80FD5F0E0
:10020000DAE4CDFBE4CCFAE4C8F922EB9FF5F0EA9E
:100210009E42F0E99D42F0E89C45F022E8600FEC38
:10022000C313FCED13FDEE13FEEF13FFD8F122E82C
:10023000600FEFC333FFEE33FEED33FDEC33FCD83C
:10024000F122E6FC08E6FD08E6FE08E6FF22E6FBF2
:1002500008E6F908E6FA08E6CBF822ECF608EDF62F
:1002600008EEF608EFF622ECF208EDF208EEF208DE
:10027000EFF222D083D082E493F608740193F6085B
:10028000740293F608740393F6740473D083D082D7
:10029000E493F208740193F208740293F208740371
:1002A00093F27404738A838982E473E4F530E53051
:1002B00025E025E0248CF8C000120232C0077452F9
:1002C0002530F8E6FFFBE4FAF9F8D0071200DED09B
:1002D0000012024BE53025E025E0248CF8C0001226
:1002E0000232780712020CD00012024BE53025E0F2
:1002F00025E0248CF8120232EC4D4E4F6076E5304A
:1003000025E025E02474F8120232E53025E025E0EE
:10031000248CF812023EC31201FB50037F0322E536
:100320003025E025E02474F812023EC000E53025B7
:10033000E025E0248CF8120232D000C3EF9BF534A4
:10034000EE9AF533ED99F532EC98F531E47FFF7EC6
:10035000FFFDFCAB34AA33A932A831C31201FB4024
:10036000037F0322E53025E02400F8E533F208E5B9
:1003700034F28015E530C39403500BE53025E024BA
:100380000CF8E4F208F27F03220530E530640360E4
:100390000302029EE4F530E53025E02406F8E2FE93
:1003A00008E2FFE53025E02400F8E2FC08E2FDD396
:1003B0009FEC9E401EE53025E02406F8E2FE08E2B0
:1003C000FFC3ED9FFFEC9EFEE48F388E37F536F5C8
:1003D000358009E4F538F537F536F535AF38AE3701
:1003E000AD36AC35780712021F8F388E378D368CBC
:1003F0003590008CE070447F03FEFDFCAB38AA37DB
:10040000A936A8351200DEE53025E025E0241EF8E7
:10041000E2FB08E2F908E2FA08E2CBF8EB2FFFEA88
:100420003EFEE93DFDE83CFC780212020CE5302579
:10043000E025E0241EF81202578033E53025E02540
:10044000E0241EF8E2FC08E2FD08E2FE08E225389E
:10045000FFEE3537FEED3536FDEC3535FC78011213
:10046000020CE53025E025E0241EF8120257E530A5
:1004700025E025E0241EF8E2FC08E2FD08E2FE0883
:10048000E2FF780712020CE53025E0240CF8EEF2CA
:1004900008EFF20530E530640360030203877F074D
:1004A000228E328F33E4F535F536F53790009FE034
:1004B000F536A3E0F537E4F534E518701690008FB3
:1004C000E0B4050FD39000A9E094009000A8E09458
:1004D00000401EE53425E0245EF8E4F208F2E5343D
:1004E00025E025E0244CF812027C00000000020503
:1004F000A8E53425E0245FF9E3700219E3701AE5FA
:100500003425E02400F8E2FE08E2FFE53425E0248B
:1005100058F8EEF208EFF28057E53425E02458F859
:10052000E2FE08E2FFE53425E02400F8E2FC08E200
:10053000FD121A7CD3EF9537EE95364033E534251E
:10054000E02400F8E2FE08E2FFE53425E02458F854
:10055000EEF208EFF2E53425E0245EF8E4F208F26A
:10056000E53425E025E0244CF812027C0000000070
:10057000E53425E02400F8E2FE08E2FFE53425E05A
:1005800025E0244CF8C000E2FB08E2F908E2FA0892
:10059000E2CBF8E4FCFDEB2FFFEA3EFEED39FDEC8B
:1005A00038FCD000120257E53425E0245EF808E25A
:1005B0002401F218E23400F20534E534C394025009
:1005C000030204A9E4F534E53425E0245FF9C3E32C
:1005D000953319E39532400205350534E534B4020C
:1005E000E6E5356402600302068574FF9000A1F021
:1005F000A3F0E4A3F0A3F0F534E53425E0245EF89D
:10060000E2FE08E2FF4E7003020685E4FCFDC00432
:10061000A905AA06AB07E53425E025E0244CF8E25D
:10062000FC08E2FD08E2FE08E2FFD0001201698E3C
:10063000388F39D39000A2E095399000A1E0953829
:100640004007E538F0A3E539F0C39000A4E0953900
:100650009000A3E095385007E538F0A3E539F0E5C0
:100660003425E02406F8E538F208E539F2E53425CA
:10067000E0245EF8E4F208F2E53425E025E0244CBD
:10068000F812027C00000000C2080534E534640260
:1006900060030205E922E4F534F533E53325E0256E
:1006A000E0244CF812027C000000000533E533B46E
:1006B00003E91217EDE4F533E53325E025E0244C9A
:1006C000F8C000E2FC08E2FD08E2FE08E2FFE533C4
:1006D00025E025E02480F812023EEF2BFFEE3AFEE3
:1006E000ED39FDEC38FCD0001202570533E533B488
:1006F00003C60534E534C3940540B7E4F533AF349D
:10070000E4FCFDFEC004A905AA06AB07E53325E01D
:1007100025E0244CF8E2FC08E2FD08E2FE08E2FFD6
:10072000D0001201698F388E378D368C35AB38AAE0
:1007300037A936A835C00074522533F8E6FFE4FC2B
:10074000FDFED0001200DE8F388E378D368C357866
:100750000712020C8F388E378D368C35E47FE87E99
:1007600003FDFCAB38AA37A936A835D31201FB40EC
:1007700030E5382418FFE53734FCFEE53634FFFD5C
:10078000E53534FFFCE53325E025E02474F812025A
:100790004BE53325E02400F87403F20874E8F28096
:1007A0001EE53325E025E02474F812026300000002
:1007B00000E53325E02400F8E537F208E538F2E5F6
:1007C0003325E025E0244CF812027C00000000E50F
:1007D0003325E0245EF8E4F208F2E533C3940350D5
:1007E00033E53325E02400F8E2FE08E2FFE5332597
:1007F000E02406F8EEF208EFF2E53325E0240CF8E9
:10080000E4F208F2E53325E025E0241EF812027C2C
:10081000000000000533E533640360030206EE22A6
:1008200085BA3953BA0F43BA10E4F533E53325E0FE
:1008300025E02480F8120263000000000533E53350
:10084000B403E975330575ABFF12199CE4F534E583
:100850003425E025E02480F8C000120232C004C034
:1008600005C006C00774982534F8E675F003A42483
:1008700096F582E4341AF583E493FB740193FA74D9
:100880000293F9120295A804A905AA06AB07D0079E
:10089000D006D005D004EF2BFFEE3AFEED39FDEC8B
:1008A00038FCD00012024B0534E534C39403409F5A
:1008B000E4F5AB12199CE4F534E53425E025E02499
:1008C00080F8C000120232C004C005C006C0077420
:1008D000982534F8E675F003A42496F582E4341ADA
:1008E000F583E493FB740193FA740293F912029571
:1008F000A804A905AA06AB07D007D006D005D004E6
:10090000C3EF9BFFEE9AFEED99FDEC98FCD0001230
:10091000024B0534E534C39403409E1533E5336040
:1009200003020836E4F534E4753810753727F536D8
:10093000F535AF38AE37AD36AC35780712021F8FBC
:10094000388E378D368C35E53425E025E02480F867
:1009500012023E1201698F388E378D368C357452F3
:100960002534F8A6070534E534B403BB8539BA222B
:10097000E4FD300420ED25E02439F582E43418F557
:1009800083E493FE740193FFED25E02434F8A6067A
:1009900008A607801EED25E02429F582E43418F529
:1009A00083E493FE740193FFED25E02434F8A6065A
:1009B00008A6070DBD02BBE4FDED25E0242AF8E200
:1009C000FE08E2FFED25E02413F9D3E39F19E39E2F
:1009D0004016ED25E02412F8E2FE08E2FFED25E0E6
:1009E000242AF8EEF208EFF2ED25E02434F8E6FED2
:1009F00008E6FFEEC313FEEF13FFED25E02413F925
:100A0000D3E39F19E39E5034ED25E02434F8E6FE4D
:100A100008E6FFED75F008A4245CF8A60608A60712
:100A2000ED25E02434F8E6FE08E625E0FFEE33F895
:100A3000ED25E0242AC8F208EFF2803CED25E02401
:100A400049F582E43418F583E493FE740193FFEDD5
:100A500025E02413F9D3E39F19E39E401BED25E025
:100A6000242AF9E3C313FE09E313FFED75F008A48C
:100A7000245CF8A60608A6070DED640260030209CF
:100A8000A9E4FDED75F008A4245CF8E6FE08E6FF95
:100A9000ED25E02430F8EEF208EFF20DBD02E4227D
:100AA00074FFF537F538E4FFFEF532E53225E02432
:100AB0003AF8E2FC08E2FDE53225E02438F8ECF2F1
:100AC00008EDF20532E532B409E17804E2FD08E20E
:100AD000784ACDF208EDF2E4F532E53225E024382B
:100AE000F8E2FC08E2FDC39538EC953750048C37EA
:100AF0008D38D3ED9FEC9E4004AE04AF050532E582
:100B000032B40AD6E538245AFDE43537FCD3EF9DDC
:100B1000EE9C4011D2097F041219039000AAEEF056
:100B2000A3EFF08002C209E4F535F536F532E5327F
:100B300025E0240CF8E2F53308E2F534C39536FFDE
:100B4000E5339535FEE4FCFD7B64FAF9F81200DE2E
:100B5000C006C007E53225E02464F582E43400F5E0
:100B600083E0FEA3E0FFFBAA06E4F9F8D007D00675
:100B7000120169E53225E02418F8EEF208EFF2AE32
:100B800033AF34E4FCFD7B64FAF9F81200DEC006F2
:100B9000C007E53225E02464F582E43400F583E003
:100BA000FEA3E0FFFBAA06E4F9F8D007D006120185
:100BB00069E53225E02412F8EEF208EFF20532E59D
:100BC0003264026003020B1E22439F04E453C6DF1B
:100BD000E5C600B5C6F375830075820775FD0DE4A3
:100BE000E5FEF4FF75830075820675FD0DE4E5FEF4
:100BF000B50704F59E8003759E0078100000D8FCB0
:100C000053C6E043C60843C68075960775970375BB
:100C1000830075820475FD0D85FE8F7583007582D6
:100C20000375FD0DE4E5FEF4FF7583007582027522
:100C3000FD0DE4E5FEB50704F59580037595837514
:100C4000BE0E5392FE9001007F007E02E4F0A3DF0F
:100C5000FCDEFA78007F00E4F208DFFC78FFE4F6BF
:100C6000D8FD7581A3020C96020000020CDBE49310
:100C7000A3F8E493A34003F68001F208DFF480298F
:100C8000E493A3F85407240CC8C333C4540F44207E
:100C9000C8834004F456800146F6DFE4800B01026D
:100CA0000408102040809015BBE47E019360BCA333
:100CB000FF543F30E509541FFEE493A360010ECFBB
:100CC00054C025E060A840B8E493A3FAE493A3F8E5
:100CD000E493A3C8C582C8CAC583CAF0A3C8C582A5
:100CE000C8CAC583CADFE9DEE780BE121A447D01A7
:100CF000E4FF1218987F01121A087F01121A2712B6
:100D00001B90121B831219C21214731218CE1219DF
:100D100037D2AF753E01E53E24FD601714602024F4
:100D2000FE602E146032147003020DBE24076003AF
:100D3000020DC1121720121254753E04020DC1D2C9
:100D4000D8E53F70FC12003E121AAE753E06020D49
:100D5000C112029B8F3E8079D3900095E094009061
:100D60000094E09400400CA3E024FFF0900094E095
:100D700034FFF0D39000A9E094009000A8E0940024
:100D8000400CA3E024FFF09000A8E034FFF0D390E3
:100D900000ABE094009000AAE094004016A3E02489
:100DA000FFF09000AAE034FFF0E07002A3E07003CF
:100DB000121551900091E004F07006900090E0044C
:100DC000F012137A120F0B8F3E753E048003753EAE
:100DD000049000A5E0B40124E4784BF6FF121B90C8
:100DE000E4F0F51CF51D00051DE51D7002051CB4A1
:100DF0002CF4E51CB401EF7F01121B901210E202EB
:100E00000D06227533077D0774017E00A833088024
:100E100005C333CE33CED8F9FFACACECFBE4EF5BCB
:100E20007003D533E3ED601D74017E00A8050880D2
:100E300005C333CE33CED8F9FFACAEECFBE4EF5BA9
:100E400070031D80E0AF337401A807088002C3332C
:100E5000D8FCF5AC7401A805088002C333D8FCFFA8
:100E6000F5AD8FAE53AACF85BA3C53BA0F43BA1033
:100E7000E4F537F536F535F53412199CE4F533749D
:100E8000982533F8E675F003A42496F582E4341A25
:100E9000F583E493740193FA740293F91202958F27
:100EA0003B8E3A8D398C38AB37AA36A935A834C376
:100EB0001201FB500C853B37853A3685393585382C
:100EC000340533E533C3940340B5AF37AE36AD35A3
:100ED000AC34780212020CE5372FF537E5363EF5D3
:100EE00036E5353DF535E5343CF534AF37AE36AD56
:100EF00035FC781012020C8FB3AF37AE36AD35AC7F
:100F000034780812020C8FB28537B143AA30853C81
:100F1000BA75AC0375ADC075AEC022E4F53075315D
:100F200008120A9012176B1212EF1217AF90008D71
:100F3000EFF012000EEF605F7F01121903AD07ACF6
:100F400006D3900095E09400900094E09400401047
:100F5000ECC4F854F0C868FCEDC4540F48FD802E72
:100F6000300811EDAE047803CEC313CE13D8F9FDCB
:100F7000AC06801AC37835E2942818E29400500E2B
:100F8000ECC4F854F0C868FCEDC4540F48FDAF053C
:100F9000AE041204918003AF312290008CE06034E3
:100FA000E4900098F0A3F0900097E004F0700690B1
:100FB0000096E004F07F05121903D3900097E09F9C
:100FC000900096E09E4014E4FF12161AE490008E02
:100FD000F07F0322E4900096F0A3F090008CE0FFF5
:100FE00090008EE06F602A12161A90008CE090003C
:100FF0008EF0784CE654F060187F0C1219039000C4
:10100000A8EEF0A3EFF09000A8E0C313F0A3E01364
:10101000F0AF3122C0E0C0F0C083C082C0D075D034
:1010200008C2CF30CD030210D730CB4720CC447854
:1010300040A6CEE6FFC39480403075F003EFA424B1
:101040004CF582E5F03415F583E493FB740193FAD3
:101050007402938B238A24F5250525E52570020566
:101060002414F912005EF5CE80097840E62522F8B6
:10107000E6F5CE30CC297840E6C394804015AB230A
:101080000525E525AA247002052414F912005EF551
:10109000CE8050784006E62522F8E6F5CE80442042
:1010A000CB41AFCE7840E6FE7028BF10028034BF3F
:1010B0002002802FBF5008784FE64401F68024BFFD
:1010C0006008784FE654FEF680197841A60F18069E
:1010D0008011EEC3940A50087840E62441F8A60F28
:1010E000784006784B7601D0D0D082D083D0F0D033
:1010F000E03220CA030211A27841E670030211A275
:10110000E4784BF6F53074412530F8E6FF74262577
:1011100030F8A60774412530F8E4F60530E530B420
:101120000AE4784BE6700320CA12E4F530742625F1
:1011300030F8E4F60530E530B40AF222E52624E082
:10114000600F24B0601224607017E4FF121A088048
:10115000107F01121A088009E4FF121AD77851A6ED
:1011600007E52654F064807049E52745286043E58B
:1011700027FE7C00E42528FFEC3EFEC3EF940AEE38
:101180009400402EE526540FFDBD0F19E4F530E51F
:101190003075F008A4245CF8A60608A6070530E51B
:1011A00030B402EB22ED75F008A4245CF8A6060822
:1011B000A60722E4FFFEEE75F008A4245CF8E6FC26
:1011C00008E6FDEE25E02419F9C3E39D19E39C40F0
:1011D0000D7401A806088002C333D8FC42070EBE76
:1011E00002D4807DEEC394025077EE75F008A424FB
:1011F0005CF8E6FC08E6FDEE25E02419F9C3E39D62
:1012000019E39C401DEE25E0241DF9C3E3940A195F
:10121000E39400400D7401A806088002C333D8FC93
:101220004207EE75F008A4246CF8E6FC08E6FDEE33
:1012300025E0241DF9C3E39D19E39C4021EE25E040
:101240002419F9C3E3940A19E394004011EE24022F
:10125000FD7401A805088002C333D8FC42070E8044
:10126000838F1822E4F531F532121A61E490008C74
:10127000F090008EF0A3F0900096F0A3F0A3F0A3FE
:10128000F09000ACF0A3F09000A8F0A3F0F521F5E9
:1012900030E53025E02464F582E43400F583E0FE97
:1012A000A3E0FF9000A0E02FF090009FE03EF0054B
:1012B00030E530B402DB90009FE0FEA3E0FF7C004D
:1012C0007D0A12008990009FEEF0A3EFF0120DF35B
:1012D000120810120686E4F530E53025E02438F8CF
:1012E0007403F20874E8F20530E530B40AEB7F0AC3
:1012F000121903900094EEF0A3EFF0121AAE22E45C
:10130000F532E53225E02406F8E2FE08E2FFE53298
:1013100025E02400F8E2FC08E2FDC39FEC9E504863
:10132000E53225E02407F8C3E29DF53418E29CF588
:1013300033FEAF34E4FCFD7B64FAF9F81200DEC042
:1013400006C007E53225E02464F582E43400F58325
:10135000E0FEA3E0FFFBAA06E4F9F8D007D00612EE
:1013600001698E358F368009E4F533F534F535F5AE
:1013700036D3E536940AE53594004002D2080532AA
:10138000E532640260030212F222E4F530E53075C2
:10139000F008A4245EFFE53025E02412F8E2FC0802
:1013A000E2FD121AC3E53075F008A42460FFE530B1
:1013B00025E0240CF8E2FC08E2FD121AC3E53075C2
:1013C000F008A42462FBC003E53025E02400F8E225
:1013D000FE08E2FFE4FCFDE53025E025E02474F89A
:1013E00012023EEF2BFFEE3AFEED39FDEC38FC78B1
:1013F0000412020CAD07AC06D007121AC30530E583
:1014000030C394024087784FE6F520227DFF80703C
:101410007864E6FE08E6FFC3781BE29F18E29E4070
:10142000107874E6FE08E6FF781FE29F18E29E50EF
:101430004F7810E2FE08E2FF780DE22FF53518E252
:101440003EF5347812E2FE08E2FF780FE22FFF1833
:10145000E23EAB07FAEB25E0FFEA33FEC3E5359F3A
:10146000E5349E50035305FAE53525E0FFE53433B6
:10147000FEC3EB9FEA9E50085305F580035305F029
:101480008D1922E4F530784CF6FF121AD78F30E52B
:1014900030BFFF06784D76068004784D76FF784E93
:1014A0007601E408F6785176FFFFEF25E02429F570
:1014B00082E43418F583E493FC740193FDEF75F036
:1014C00008A4245CF8A60408A605EF75F008A42477
:1014D0005EF8E4F608F6EF75F008A42460F8E4F688
:1014E00008F6EF75F008A42462F8E4F608F60FBFDA
:1014F00003B875224C22C0E0C0F0C083C082C0D0C7
:1015000075D000C000C004C005C006C007C28D75FC
:101510008CD8758AF0051FE51F7002051EAE1EFFF0
:101520007C007D64120089ED4C7021900090E0FEFB
:10153000A3E0FFD3940AEE94004006A3EEF0A3EFDD
:10154000F0900090E4F0A3F0F51EF51FD007D00650
:10155000D005D004D000D0D0D082D083D0F0D0E05D
:1015600032E4FBEB25E025E0248CF8120232EF2474
:1015700018FFEE34FCFEED34FFFDEC34FFFCEB25F0
:10158000E025E02474F812024BEB25E02400F87407
:1015900003F20874E8F2EBC394035017EB25E02440
:1015A0000CF8E4F208F2EB25E02406F87403F208E4
:1015B00074E8F20BBB03ACE4FBEB25E02438F874D1
:1015C00003F20874E8F20BBB0AEF2208980102004C
:1015D000FFFFFFFFFF04A000000000604A0064025C
:1015E00008012C006400640064006400640064016D
:1015F00002040805060708000000000000000000C3
:1016000000000000000000000000000000000000DA
:1016100000000000000000000000000000000000CA
:10162000000000000000000000009000A5E07055E0
:1016300004F0E4FEFDFC7401A804088002C333D862
:10164000FCF9FB90008EE05BB50313EC2404FA7404
:1016500001A802088002C333D8FC42068003E94295
:1016600006EF5BB50305E942058011EC2404FB7429
:1016700001A803088002C333D8FC42050CBC02B6A3
:10168000EE5D784CF622C0E0C0F0C083C082C0D0CE
:1016900075D01053B9FD753D007498253DF8E67579
:1016A000F003A42496F582E4341AF583E4937401DC
:1016B00093FA740293F9120295E53D25E025E024A2
:1016C00080F812024B053DE53DC3940340CB753FC6
:1016D00000D0D0D082D083D0F0D0E032FE0000FE27
:1016E0000008FE0006FE000EFE000CFE0014FE00C8
:1016F00012FE001AFE0018FE002000008000008884
:1017000000009000009800001801008D01008C017D
:10171000008EFE001EFE002A0100900100AA0100BA
:10172000A50100A801007C010084FE0030FE005EDF
:10173000E4FFFE74982EF8E69018599342070EBE07
:1017400003F1EF42D4EF42F4EF42E4EFF452DC75E0
:10175000AA3B75BA0C43BA4043B92053B9BF8FB402
:10176000E4F5B375B24E75B12075BBFF75A950F5A0
:10177000AB75AC0375ADC075AEC0227818E2FE083B
:10178000E2FF8E32F5337D01ED25E02418F8E2FA10
:1017900008E2FBC39533EA953250048A328B33D387
:1017A000EB9FEA9E4004AE02AF030DBD02DA78362D
:1017B000E532F208E533F27834EEF208EFF2221265
:1017C00009601211A31213FC120003121862900098
:1017D0008CE0700D851833E5195233E51A523380C9
:1017E00003851B339000AAE07002A3E07009AF33B9
:1017F00012196B8F328003E4F532AF322212199C3A
:10180000E4F53974982539F8E675F003A42496F5C3
:1018100082E4341AF583E493740193FA740293F921
:10182000120295E53925E025E02480F812024B05E7
:1018300039E539C3940340CB22003C002D0032002F
:101840003200320032003200320032003200320008
:101850003200320032003200320064006400320094
:1018600032003200320032003201020408102040FF
:10187000800FE4FFFEEE75F008A4245DF8E624FB7B
:10188000FD18E634FFFCEE25E02413F9C3E39D19AF
:10189000E39C400D7401A806088002C333D8FC42C3
:1018A000070EBE02D08F1B22E4FE7C0274982CF837
:1018B000E69018599342060CBC03F1EF6005EE4226
:1018C000D48004EEF452D4EEF4FF52F4EE42E4ED90
:1018D0006005EE42EC8003EF52ECEF52DC227E001A
:1018E0007F7CE4FDED25E024E8F582E43419F583FE
:1018F000E493F4601DED25E024E9F582E43419F564
:1019000083E493FCEF2DF582E43EF583ECF00DBD0E
:1019100010D222753900753A7C7B017A00BFFF0531
:101920007F017E0022E53A2FF582E43539F583E028
:101930007A00FB900092E0FCA3E0FDAF037E001272
:101940000077AA06AB072243F80875CD4053CC7F39
:1019500043CC4043CC2043CC1043CC0453CCFD4378
:10196000CB0243CB0153CBBF43E80853E5FC43E331
:101970000243F50343900343ED0322A907E4FDFC72
:1019800074017E00A804088005C333CE33CED8F995
:10199000FFE9FBE4EF5B600D7401A804088002C35B
:1019A00033D8FC42050CBC02D7AF052275BF0F002F
:1019B0000000000000000000000000000000000027
:1019C00000D2D853B9FD43B901E5B930E1FBE4F5E4
:1019D000BF22438901C28DD2A953B8FDE4F51EF59B
:1019E0001F900090F0A3F0A3F0A37464F0758CD85E
:1019F000758AF0D28CD2AF220002010102010301EC
:101A00000402050606060702080A09020A020B2854
:101A10000C010D030E01FF01E4FE7D0274982DF808
:101A2000E69018599342060DBD03F1EF6004EE42B3
:101A30008022EEF4528022EF600543D504800353E8
:101A4000D5FB53F5FB53E5FB43E30443ED04E4907E
:101A500000A5F022E4F5E3439F10439F02FF0FBF70
:101A6000FFFC539FEF75BE0EE4F5BFF5B975927696
:101A70002253BAFEE5B920E004E53F6005E5B93040
:101A8000E1FBE4F5BF53B9FE53B9FD22AB07AA064B
:101A9000D3EB9DEA9C4007EB9DFFEA9CFE22C3ED41
:101AA0009BFFEC9AFE22FF1AEBFF1AFEFF1B11FFB1
:101AB0001B24FF1B37FF1B4AFF1B5DFF1B7075BFFD
:101AC0000F43B92053B9FD43BA01753F0143B90132
:101AD000D2D822AB07AF04AE05C2AFA803A607E871
:101AE00004F8A606D2AF22E4FFF582F5837420FE47
:101AF000E493F42FFFA3EEB583F62253B9EF78A158
:101B0000A6B708A6B608A6B578A01202322253B925
:101B1000EF78A1A6EB08A6EA08A6E978A01202329F
:101B20002253B9EF78A1A6F308A6F208A6F178A08F
:101B30001202322253B9EF78A1A6FB08A6FA08A632
:101B4000F978A01202322243B91078A1A6B708A6EC
:101B5000B608A6B578A01202322243B91078A1A621
:101B6000EB08A6EA08A6E978A01202322243B910CF
:101B700078A1A6F308A6F208A6F178A012023222F4
:101B800043B91078A1A6FB08A6FA08A6F978A01216
:101B9000023222C2DA53D80F43D8D0D2D8D2D922B7
:101BA000EF6003D29222C29222FFFFFFFFFFFFFFEE
:00000001FF
